:10007400C0E0C0F0C083C082C0D075D008438CDC1F
:10008400858C8C05231200F4D0D0D082D083D0F09C
:03009400D0E03287
:10009700D2AFD2A9438901858989D28C7518FFE42B
:1000A700F523751412F513F5117524FFF515751F52
:1000B70012752001752112752202F526751B4075F0
:0800C7001C40751D40751E4030
:1000CF00E5236480B48100500512012E80F2E4F51F
:1000DF002312016B12019C1202AA1201B2120278B2
:0500EF0012028780DB16
:0900F4000510E510B46400403071
:1000FD00E4F5104315057517320511E511B43C00F3
:02010D00401E92
:0F010F00E4F5114315020513E513B43C00400F4E
:0C011E00E4F5130514E514B418004003C8
:04012A00E4F51422C2
:0B012E00751A087524FFE4F533F53462
:10013900E51AF4FAE5185AF5B0E534241BF8E6F4A3
:10014900F590E4FE7F051202B37590FFE5B020E457
:1001590003853424E51AC313F51A0534E534B404C8
:02016900CF22A3
:10016B0075F00AE51384E5F02427F8861B75F00A71
:10017B00E513842427F8861C75F00AE51484E5F052
:10018B002427F8861D75F00AE514842427F8861EAB
:01019B002241
:05019C00E51530E21042
:0601A1001517E5176007C9
:0B01A700431C80431D80225315FB22E7
:0501B200E524F46028C3
:0501B700E51520E7231F
:1001BC00431580752532E524600A14600B14600C1D
:0401CC0014600D228C
:1001D000120233221201F9221201EB221201E02253
:0B01E0000514E514B41803E4F5142224
:0E01EB000513E4F511E513B43C03E4F513220B
:0701F9000526E526B40116FE
:1002000085141F851320751B00751C68751D787576
:060210001E7112025D22C6
:07021600E4F52612021D228F
:10021D00851421851322751B63751C63751D7875F7
:06022D001E7112025D22A9
:0A023300E518F4447FF51820E710E9
:10023D00751B00751C00751D68751E7812025D22F8
:10024D00751B00751C63751D63751E7812025D228A
:10025D00E4F531F53212012E0532E5327002053129
:0B026D00E531B407F0E532B4D0EB221D
:05027800E51530E70967
:0A027D001525E525700353157F22B7
:05028700E51530E01D4B
:10028C005315FEE514B51F08E513B5200375187F4B
:0E029C00E514B52108E513B522037518FF22FD
:0902AA00E51EB43F03751E00229D
:1002B300E4FCFD8EF0B2F7EC6480B5F004EDB50715
:0B02C3000050070DED70EC0C80E922EC
:0C02CE0028273F0C765E4D5B7B0E7F5FA7
:03000B000200747C
:0300000002000EED
:10000E00758135E4787FF6D8FD9002CEE4937002C8
:10001E00804EC31392D5C31392D1FFA3E493F8B0CD
:10002E00D5402130D505E4A393F5A0E420D102A359
:10003E009320D507F608DFF3A380D1F208B800F6B7
:10004E0005A080F2E8030303541F2420F9E85407A7
:10005E00F8E4D333B80002800333D8FD47F780D8D5
:06006E0075A0FF020097DF
:0102DA000023
:00000001FF
